:020000040000FA
:04000000D3303A2897
:040004000034003490
:08000800A000030EA100831209
:100010008B1C32288B1032181428B21C3228643002
:10002000010203183128182800001628172818285C
:1000300019281A281B281C281D281E281F283210A2
:10004000B214A810031005190314AA0DA90DA80DC8
:10005000B10B322832152A08AF002908AE00280853
:10006000AD00B21081010B11210E8300A00E200EF5
:02007000090085
:0C007400203084008001840A80300402E7
:10008000031C3C281230B1008621850187018316AC
:100090000C308505870183128316051483128501B0
:1000A00087010730990000309A00103083168E00C7
:1000B0008312603083168F00831200308316910004
:1000C0009F008312C8308316810083123130900064
:1000D000003083168C00831210308B00BD1B7228F9
:1000E000851D0027DA2181018E018F010B118B10F4
:1000F0000B108C018B178A203219A020B40B882892
:10010000031085190314BA0DF0303A0203191221B5
:10011000C0237B286400321808000B1D08000B1157
:10012000B21032141230B100051D9B28331483160F
:10013000011383120800331083160117831208007D
:1001400032110130B7008B132030370783169B0024
:100150001C141A088312A400A500C030A506103094
:10016000370783169B001C141A088312A300003063
:10017000370783169B001C141A088312A2008B17E2
:10018000331CC82822090339A200A309A409A50920
:1001900022082D02031D0C2923082E02031D0C2901
:1001A00024082F02031D0C2901303702031DDB2810
:1001B0003E143F14BA2102303702031DE228BE1458
:1001C0003F14BE2103303702031DE9283E153F14BA
:1001D000C22104303702031DF028BE153F14C6218A
:1001E00005303702031DF7283E163F14CA2106309A
:1001F0003702031DFE28BE163F14CE2107303702FA
:10020000031D05293E173F14D22108303702031D74
:100210000C29BE173F14D621B70A0930370203183C
:100220000800A3283D1C08000130B600B400B5004A
:10023000B70085018701B2138A20B40B2E29031061
:1002400085190314BA0DF0303A0203195529B51F68
:100250008512B50B2E299630B5005F21321D1C2961
:100260003211331C38292D090339AD00AE09AF090D
:100270002F1CB2132F1C1C29B21B1C292E181C2941
:10028000B2178B1320303707BC002F08BB00712139
:1002900010303707BC002E08BB0071210030370733
:1002A000BC002D08BB0071218B1785018701B70A9F
:1002B000B60109303702031C1C29DA21080037086F
:1002C000B6080319B600031908008516B60308001E
:1002D0003F1C08003F101030BC003E08BB007121DD
:1002E00008008B133B0883161C159A0083123C08E8
:1002F00083169B0055309D00AA309D009C1464001D
:100300009C187F291C1183128B170800831600305C
:100310009B001C141A088312BD00831610309B002A
:100320001C141A088312BE0000309500603084004F
:100330008B13831604089B001C141A0883128B1756
:100340008000840A68300402031C98296430D500B8
:10035000E724DC006430D500EC24DD006430D500F7
:10036000F124DE006430D500F624DF003C30F200DA
:10037000F30008000130E800072208000230E8001E
:10038000072208000430E800072208000830E800CF
:10039000072208001030E800072208002030E8009B
:1003A000072208004030E800072208008030E800FB
:1003B00007220800F0178B13831670309B001C1463
:1003C0001A0883128B17E80007228B1383167130EB
:1003D0009B001C141A0883128B17E80007228B134A
:1003E000831672309B001C141A0883128B17E800C6
:1003F00007228B13831673309B001C141A08831278
:100400008B17E80007220430F100F0130800E80819
:1004100003190800681C142A6730D500E724D100AE
:100420006830D500E724D200E81C1E2A6730D500CA
:10043000EC24D1006830D500EC24D200681D282AB5
:100440006730D500F124D1006830D500F124D20006
:10045000E81D322A6730D500F624D1006830D50077
:10046000F624D200681E3C2A6A30D500E724D10069
:100470006B30D500E724D200E81E462A6A30D5004A
:10048000EC24D1006B30D500EC24D200681F502A38
:100490006A30D500F124D1006B30D500F124D200B0
:1004A000E81F5A2A6A30D500F624D1006B30D500F7
:1004B000F624D200F016D11A8B2A511B8B2A511C1C
:1004C0006A2ADC1FF0125C1F8B2A501C8B2AC01B6F
:1004D0008B2A0800D11C752ADD1FF0125D1F8B2AA4
:1004E000D01C8B2AC11B8B2A0800511D802ADE1FBD
:1004F000F0125E1F8B2A501D8B2AC21B8B2A08000C
:10050000D11D8B2ADF1FF0125F1F8B2AD01D8B2A73
:10051000C31B8B2A0800F01EA12AF01BA12A511828
:100520007030D118713051197230D11973308B136A
:1005300083169B001C141A0883128B176802031978
:100540000800D11ABE2A511BBE2A7010511CAC2AB9
:100550005014541F70145417D11CB22AD014D41F35
:100560007014D417511DB82A5015D41E7014D41607
:10057000D11DBE2AD015541E70145416511CC62A03
:10058000511A5016D11AC017511B5012D11CCE2A25
:10059000511AD016D11AC117511BD012511DD62A8B
:1005A000511A5017D11AC217511B5013D11DDE2AF0
:1005B000511AD017D11AC317511BD013F01FE52AB7
:1005C000D11A0800511B0800E92AD11A462B511BE9
:1005D000462B6530D500521AE724D21AEC24521B60
:1005E000F124D21BF6245118C400D118C5005119AA
:1005F000C600D119C7006630D500521AE724D21AB6
:10060000EC24521BF124D21BF6245118CC00D11833
:10061000CD005119CE00D119CF0052085118D70082
:10062000D118D8005119D900D119DA000430701846
:100630003230F01B32305118C800D118C90051199E
:10064000CA00D119CB0051185C14D1185D1451198E
:100650005E14D1195F14F01F3E2B511C312B440343
:10066000C000D11C352B4503C100511D392B460359
:10067000C200D11D3D2B4703C30008005118C00123
:10068000D118C1015119C201D119C30151187030DB
:10069000D118713051197230D1197330BC0068080B
:1006A000E900BB007121BE0108007013851A7017A4
:1006B000851254188516071407108512D41885164C
:1006C0000714071085125419851607140710851290
:1006D000D4198516071407108512541A85160714A5
:1006E00007108512D41A8516071407108512541B9B
:1006F0008516071407108512D41B851607140710DA
:100700000516051285148512701B85160800FD015B
:100710000730FF007B08FE0C0318922BFF0B8B2B7E
:10072000FB0100340310972BFE0C0318FB07FB0C96
:10073000FD0CFF0B942BFB0CFD0C0034940193017A
:10074000083095008B138E018F018B17D613560836
:10075000FB007508F51BFF3CFE00FE138723FD0D13
:100760007B0DF51FD607F51BD602560876079300BA
:0A0770000318141409309500080066
:1007800002300F02031C0800BF27F4080319E52BF1
:100790006E30D5007419F124F419F6243D18D42BC9
:1007A0007418E724F418EC24E8006818BA21E81853
:1007B000BE216819C221E819C621681ACA21E81A9F
:1007C000CE21681BD221E81BD62107118710871183
:1007D00007120730F10503308A0071088207F42BF5
:1007E0002C2C642C9C2CD42C0715501CE02C40087D
:1007F000D500571AE724D71AEC24571BF124D71B2E
:10080000F624D6005709F038D40557080F39D61BFF
:10081000D4046108F5006008F6005C1C9E23C80B38
:10082000E02C4C085C180530C8005C1CC00A5C1049
:1008300044084002031CE02CC01B222C501E222C1A
:10084000C001E02C5012DC1854135C1950105C1DD0
:10085000C0035C1DC017E02C8714D01CE02C41089D
:10086000D500581AE724D81AEC24581BF124D81BB9
:10087000F624D6005809F038D40558080F39D61B8D
:10088000D4046308F5006208F6005D1C9E23C90BC2
:10089000E02C4D085D180530C9005D1CC10A5D10D3
:1008A00045084102031CE02CC11B5A2CD01E5A2CB7
:1008B000C101E02CD012DD18D4135D19D0105D1DDC
:1008C000C1035D1DC117E02C8715501DE02C4208A7
:1008D000D500591AE724D91AEC24591BF124D91B45
:1008E000F624D6005909F038D40559080F39D61B1B
:1008F000D4046508F5006408F6005E1C9E23CA0B4C
:10090000E02C4E085E180530CA005E1CC20A5E105C
:1009100046084202031CE02CC21B922C501F922C52
:10092000C201E02C5013DE18D4125E1950115E1D66
:10093000C2035E1DC217E02C0716D01DE02C430831
:10094000D5005A1AE724DA1AEC245A1BF124DA1BD0
:10095000F624D6005A09F038D4055A080F39D61BA8
:10096000D4046708F5006608F6005F1C9E23CB0BD5
:10097000E02C4F085F180530CB005F1CC30A5F10E6
:1009800047084302031CE02CC31BCA2CD01FCA2CEF
:10099000C301E02C5012DF1854125F19D0115F1DF3
:1009A000C3035F1DC317E02C5523851ED92C851268
:1009B000E02CE9080319E02C85160310E90CE02C63
:1009C000F10A053071020318F1018F0108000530AA
:1009D0008A00D5135508820005308A00D5175508BE
:1009E000820006308A00D5135508820006308A003E
:0609F000D5175508820036
:100A00000034013403340434053406340834093422
:100A10000A340B340D340E340F34113412341334C1
:100A2000143416341734183419341B341C341D3460
:100A30001E342034213422342434253426342734FF
:100A400029342A342B342C342E342F34303432349D
:100A50003334343435343734383439343A343C343C
:100A60003D343E344034C134C234C334C534C6345A
:100A7000C734C834CA34CB34CC34CD34CF34D0347A
:100A8000D134D334D434D534D634D834D934DA3418
:100A9000DB34DD34DE34DF34E134E234E334E434B7
:100AA000E634E734E834E934EB34EC34ED34EE3456
:100AB000F034F134F234F434F534F634F734F934F4
:100AC000FA34FB34FC34FE34C4346434013401346D
:100AD0001134003401342134003400340134003442
:100AE0000034003400340034003400340034003466
:100AF0000034003400340034003400340034003456
:100B0000FF34FE34FC34FB34FA34F934F734F63471
:100B1000F534F434F234F134F034EE34ED34EC34B2
:100B2000EB34E934E834E734E634E434E334E234F3
:100B3000E134DF34DE34DD34DB34DA34D934D83434
:100B4000D634D534D434D334D134D034CF34CD3476
:100B5000CC34CB34CA34C834C734C634C534C334B7
:100B6000C234C1343F343E343D343C343A343934F9
:100B700038343734353434343334323430342F3439
:100B80002E342C342B342A3429342734263425347B
:100B900024342234213420341E341D341C341B34BC
:100BA00019341834173416341434133412341134FD
:100BB0000F340E340D340B340A340934083406343F
:100BC0000534043403340134C4346434013402344D
:100BD000123400340234223400340034103400342F
:100BE0000034003400340034003400340034003465
:100BF0000034003400340034003400340034003455
:100C0000803413341E3426342C34313436343934A1
:100C10003D34403442344534473449344B344C3409
:100C20004E3450345134533454345534563458348B
:100C300059345A345B345C345D345E345F34603430
:100C400060346134623463346434643465346634EB
:100C5000663467346834683469346A346A346B34AF
:100C60006B346C346C346D346D346E346F346F347B
:100C70006F3470347034713471347234723473344C
:100C8000733474347434743475347534763476341F
:100C900076347734773477347834783478347934F8
:100CA00079347A347A347A347B347B347B347B34D1
:100CB0007C347C347C347D347D347D347E347E34AD
:100CC0007E347E347F347F34C4346434013404345D
:100CD0001434003404342434003400340234003436
:100CE0000034003400340034003400340034003464
:100CF0000034003400340034003400340034003454
:100D000080340034003401340234033404340634B3
:100D100008340A340C340E341134143417341A34B1
:100D20001D342134243428342C342F3433343734D4
:100D30003B343F34433447344B344F3452345634CD
:100D40005A345D346134643467346A346D347034D9
:100D500072347434763478347A347B347C347D3431
:100D60007E347E347E347E347E347D347C347B34F9
:100D70007A34783476347434723470346D346A343E
:100D80006734643461345D345A34563452344F34E9
:100D90004B34473443343F343B34373433342F34CB
:100DA0002C342834243421341D341A3417341434A8
:100DB00011340E340C340A34083406340434033449
:100DC0000234013400340034C4346434013408344F
:100DD000183400340834283400340034203400340B
:100DE0000034003400340034003400340034003463
:100DF0000034003400340034003400340034003453
:100E00003D1C080072147314F1011430B6008512F1
:100E10000730F10507308A0071088207162F242F4A
:100E2000272F372F3A2F4A2F4D2F5D2F6108F500BE
:100E30006008F6000715871087110712D4015414B3
:100E400054175523D601602F7F30D600602F7508C8
:100E5000E1007608E0006308F5006208F60007117B
:100E60008714D401D414D4175523D601602F7F30B2
:100E7000D600602F7508E3007608E2006508F500EB
:100E80006408F60087108715D4015415D41655232D
:100E9000D601602F7F30D600602F7508E5007608F8
:100EA000E4006708F5006608F60087110716D4010C
:100EB000D41554165523D601602F7F30D600602FED
:100EC000741A892F7118692F7419F60A7418F603A9
:100ED0006D2F7419F50A7418F50350307418F20068
:100EE0007419F300C8307602C8300318F600503089
:100EF00076025030031CF600F51F842F87307502F0
:100F00008730031CF500892F6430750264300318A4
:100F1000F5007F30D600711CD6019E23F001BF275B
:100F2000741C942F731B7416741D982F721B7416E7
:100F3000741E9D2FF10AF119AE2F8512B60BA52F45
:100F400085163C3071180A30B60064000A300F0272
:100F5000031CA52F8F01741A082F602F7508E70056
:100F60007608E600603084000408BC000008BB007E
:100F70007121840A68300402031CB42F0800F401B4
:100F80000A30851DF2078519F202783072020319C2
:100F9000741479300318F200153072020319F41436
:100FA0001430031CF2000A30051CF3070518F30285
:100FB000783073020319741579300318F300153073
:0E0FC00073020319F4151430031CF30008002B
:084000000B000300060009009B
:02400E00CC33B1
:10420000010003000300030003000200020002009B
:1042100002000000000000000000FF00FF00FF009F
:10422000000000000000000000000000000000008E
:104230000000C000C000C000C000FF00FF00FF0081
:104240000100C300F300CF00FF00C300F300CF0064
:10425000FF00C300F300CF00FF00FF00FF00FF00DE
:104260004000FF00FF00FF00FF00FF00FF00FF0015
:10427000FF00FF00FF00FF00FF00FF00FF00FF0046
:10428000FF00FF00FF00FF00FF00FF00FF00FF0036
:10429000FF00FF00FF00FF00FF00FF00FF00FF0026
:1042A000FF00FF00FF00FF00FF00FF00FF00FF0016
:1042B000FF00FF00FF00FF00FF00FF00FF00FF0006
:1042C0007D00D4007D00D4007D00D4007D00D400AA
:1042D000FF00FF00FF00FF00FF00FF00FF00FF00E6
:1042E0000000000000000000FF00FF00FF00FF00D2
:1042F000FF00FF00FF00FF00FF00FF00FF00AA001B
:00000001FF
